:020000040000FA
:0408000030EF05F0E0
:1008100003B23DEF04F0F2B458EF04F09EB060EF85
:1008200004F09EB268EF04F0F2A81AEF04F0F2B2FE
:100830001CEF04F00EEF05F0CD90F29207BC078E8E
:10084000078C9EA029EF04F00101463F29EF04F038
:10085000472B07AE34EF04F0CECF51F1CFCF52F19A
:1008600046C153F147C154F1CF6ACE6A0101466BCC
:10087000476B9E90CD800EEF05F00392030103EECF
:1008800000F080517F0BE92604C0EFFF802B8151DF
:10089000805D700BD8A48B8200008051815D700B4D
:1008A000D8A48B9281518019D8B407900EEF05F02F
:1008B000F2940101383F0EEF05F0392B0EEF05F0F1
:1008C0009E900101463F0EEF05F0472B0EEF05F01D
:1008D0009E92C3CF48F1C4CF49F1C28207B492EFD0
:1008E00004F03AC13EF13BC13FF13CC140F13DC192
:1008F00041F151C155F152C156F153C157F154C1A3
:1009000058F1010148514E2749514F23E86A5023BD
:100910000D2E92EF04F04FC14AF150C14BF14E6BD6
:100920004F6B506B0201002F0EEF05F03C0E006F75
:1009300001015D67A3EF04F05E67A3EF04F05F675A
:10094000A3EF04F06067A7EF04F0D7EF04F061C1F4
:1009500000F162C101F163C102F164C103F101015F
:10096000010E046F000E056F000E066F000E076F7C
:1009700009EC11F000C161F101C162F102C163F142
:1009800003C164F10067CCEF04F00167CCEF04F021
:100990000267CCEF04F00367D7EF04F05DC161F1AB
:1009A0005EC162F15FC163F160C164F10E80D57E0A
:1009B000D5BE32D0D6CF3AF1D7CF3BF138C13CF1DA
:1009C000E86AE8CF3DF1010147A7F2EF04F0079C88
:1009D000079E0101000E516F600E526F3D0E536F66
:1009E000080E546F01013ABF02EF05F03B6702EFBA
:1009F00005F03C6702EF05F03D6702EF05F0F28875
:100A000007EF05F0F298516B526B536B546BD76A3A
:100A1000D66A0101386B396B0EEF05F002C0E0FFBA
:100A2000005001C0D8FF1000A6B214EF05F00CC0B2
:100A3000A9FF0BC0A8FFA69EA69CA684F29E550EF9
:100A4000A76EAA0EA76EA682F28EA694A6B226EF75
:100A500005F01200A96EA69EA69CA680A8501200C2
:100A6000076A0E6A0F010E0EC16E860EC06E030E6F
:100A7000C26E0F01896A110E926E080E8A6EF10E17
:100A8000936E8B6A800E946EF18E0D6A01014E6B2F
:100A90004F6B506B4A6B4B6B0F01280ED56EF28A71
:100AA000B00ECD6E9D800101516B526B536B546B38
:100AB000556B566B576B586B596B5A6B5B6B5C6B1A
:100AC000079C079E760ECA6E9D8202013C0E006F47
:100AD000CC6A160E2AEC05F0E8CF00F1170E2AECCE
:100AE00005F0E8CF01F1180E2AEC05F0E8CF02F18D
:100AF000190E2AEC05F0E8CF03F1010103AF9BEFDB
:100B000005F000EC12F0160E0C6E00C10BF014ECA8
:100B100005F0170E0C6E01C10BF014EC05F0180E69
:100B20000C6E02C10BF014EC05F0190E0C6E03C133
:100B30000BF014EC05F000C15DF101C15EF102C1E2
:100B40005FF103C160F100C161F101C162F102C155
:100B500063F103C164F11A0E2AEC05F0E8CF00F14D
:100B60001B0E2AEC05F0E8CF01F11C0E2AEC05F073
:100B7000E8CF02F11D0E2AEC05F0E8CF03F10101E8
:100B800003AFF1EF05F000EC12F01A0E0C6E00C18D
:100B90000BF014EC05F01B0E0C6E01C10BF014EC05
:100BA00005F01C0E0C6E02C10BF014EC05F01D0ECE
:100BB0000C6E03C10BF014EC05F01A0E2AEC05F0D4
:100BC000E8CF00F11B0E2AEC05F0E8CF01F11C0E76
:100BD0002AEC05F0E8CF02F11D0E2AEC05F0E8CF73
:100BE00003F100C165F101C166F102C167F103C102
:100BF00068F1240EAC6E900EAB6E240EAC6E080E37
:100C0000B86E000EB06E1F0EAF6E0401806B816B6C
:100C10000F01900EAB6E0F019D8A0301806B816BFB
:100C2000A26B8B9207900001F28EF28C07B0CDEF91
:100C30000EF00EB012EF0AF00301805181197F0B04
:100C4000D8B4CDEF0EF013EE00F081517F0BE1260A
:100C5000812BE7CFE8FFE00BD8B4CDEF0EF023EE09
:100C600082F0A2511F0BD926E7CFDFFFA22BDF5066
:100C7000780AD8A4CDEF0EF0078061C100F162C1FF
:100C800001F163C102F164C103F10101040E046FBB
:100C9000000E056F000E066F000E076F09EC11F0D5
:100CA00000AF5CEF06F00101030E616F000E626F92
:100CB000000E636F000E646F03018251720AD8B494
:100CC00012EF0AF08251520AD8B412EF0AF08251A0
:100CD000630AD8B48DEF0BF08251690AD8B4E7EFFC
:100CE00007F082517A0AD8B4FAEF08F08251490A23
:100CF000D8B486EF07F08251500AD8B4A4EF06F0BA
:100D00008251700AD8B4E7EF06F08251540AD8B481
:100D100012EF07F08251740AD8B458EF07F0C2EF0F
:100D20000BF0040114EE00F080517F0BE12682C429
:100D3000E7FF802B12000D0E826F91EC06F00A0E79
:100D4000826F91EC06F0120083C31EF184C31FF181
:100D500085C320F186C321F187C322F188C323F123
:100D600089C324F18AC325F18BC326F18CC327F1F3
:100D700001014DEC12F0C5EC11F0160E0C6E00C125
:100D80000BF014EC05F0170E0C6E01C10BF014EC17
:100D900005F0180E0C6E02C10BF014EC05F0190EE4
:100DA0000C6E03C10BF014EC05F000C15DF101C144
:100DB0005EF102C15FF103C160F100C161F101C1E7
:100DC00062F102C163F103C164F186EF07F083C3EE
:100DD0001EF184C31FF185C320F186C321F187C3AF
:100DE00022F188C323F189C324F18AC325F18BC37F
:100DF00026F18CC327F101014DEC12F0C5EC11F086
:100E000000C15DF101C15EF102C15FF103C160F19A
:100E100000C161F101C162F102C163F103C164F17A
:100E200086EF07F083C31EF184C31FF185C320F151
:100E300086C321F187C322F188C323F189C324F13A
:100E40008AC325F18CC326F18DC327F101014DEC36
:100E500012F0C5EC11F00101000E046F000E056FD9
:100E6000010E066F000E076F18EC11F01A0E0C6ED3
:100E700000C10BF014EC05F01B0E0C6E01C10BF061
:100E800014EC05F01C0E0C6E02C10BF014EC05F016
:100E90001D0E0C6E03C10BF014EC05F000C165F1E2
:100EA00001C166F102C167F103C168F186EF07F085
:100EB00083C31EF184C31FF185C320F186C321F1D2
:100EC00087C322F188C323F189C324F18AC325F1A2
:100ED0008CC326F18DC327F101014DEC12F0C5EC56
:100EE00011F00101000E046F000E056F010E066F78
:100EF000000E076F18EC11F000C165F101C166F139
:100F000002C167F103C168F186EF07F0160E2AEC03
:100F100005F0E8CF00F1170E2AEC05F0E8CF01F15B
:100F2000180E2AEC05F0E8CF02F1190E2AEC05F0B4
:100F3000E8CF03F1A3EC11F0CFEC0FF00401730E36
:100F4000826F91EC06F004012C0E826F91EC06F09A
:100F50005DC100F15EC101F15FC102F160C103F149
:100F6000A3EC11F0CFEC0FF00401730E826F91EC43
:100F700006F004012C0E826F91EC06F01A0E2AEC9A
:100F800005F0E8CF00F11B0E2AEC05F0E8CF01F1E7
:100F90001C0E2AEC05F0E8CF02F11D0E2AEC05F03C
:100FA000E8CF03F1DCEC0BF004012C0E826F91EC26
:100FB00006F065C100F166C101F167C102F168C1C7
:100FC00003F1DCEC0BF09BEC06F0C2EF0BF004013C
:100FD000690E826F91EC06F004012C0E826F91EC89
:100FE00006F00101040E006F000E016F000E026F8B
:100FF000000E036FA3EC11F020C182F40401300E47
:10100000822791EC06F021C182F40401300E822780
:1010100091EC06F022C182F40401300E822791EC9B
:1010200006F023C182F40401300E822791EC06F011
:1010300024C182F40401300E822791EC06F025C110
:1010400082F40401300E822791EC06F026C182F46E
:101050000401300E822791EC06F027C182F40401CE
:10106000300E822791EC06F004012C0E826F91EC79
:1010700006F00101030E006F000E016F000E026FFB
:10108000000E036FA3EC11F020C182F40401300EB6
:10109000822791EC06F021C182F40401300E8227F0
:1010A00091EC06F022C182F40401300E822791EC0B
:1010B00006F023C182F40401300E822791EC06F081
:1010C00024C182F40401300E822791EC06F025C180
:1010D00082F40401300E822791EC06F026C182F4DE
:1010E0000401300E822791EC06F027C182F404013E
:1010F000300E822791EC06F004012C0E826F91ECE9
:1011000006F00101110E006F000E016F000E026F5C
:10111000000E036FA3EC11F020C182F40401300E25
:10112000822791EC06F021C182F40401300E82275F
:1011300091EC06F022C182F40401300E822791EC7A
:1011400006F023C182F40401300E822791EC06F0F0
:1011500024C182F40401300E822791EC06F025C1EF
:1011600082F40401300E822791EC06F026C182F44D
:101170000401300E822791EC06F027C182F40401AD
:10118000300E822791EC06F004012C0E826F91EC58
:1011900006F0200EF86EF76AF66A04010900F5CF32
:1011A00082F491EC06F00900F5CF82F491EC06F0A0
:1011B0000900F5CF82F491EC06F00900F5CF82F436
:1011C00091EC06F00900F5CF82F491EC06F00900ED
:1011D000F5CF82F491EC06F00900F5CF82F491ECA2
:1011E00006F00900F5CF82F491EC06F09BEC06F0D6
:1011F000C2EF0BF08351630AD8A4C2EF0BF0845105
:10120000610AD8A4C2EF0BF085516C0AD8A4C2EFD2
:101210000BF08651410A42E08651440A1BE0865198
:10122000420AD8B461EF09F08651350AD8B44BEFC1
:101230000DF08651360AD8B49FEF0DF08651370A6B
:10124000D8B407EF0EF08651380AD8B465EF0EF027
:10125000C2EF0BF00798079A04017A0E826F91ECA7
:1012600006F00401780E826F91EC06F00401640E22
:10127000826F91EC06F081A845EF09F00401550E4C
:10128000826F91EC06F04AEF09F004014C0E826F78
:1012900091EC06F09BEC06F0C2EF0BF00788079A82
:1012A00004017A0E826F91EC06F00401410E826F08
:1012B00091EC06F00401610E826F91EC06F03BEFB9
:1012C00009F00798078A04017A0E826F91EC06F004
:1012D0000401420E826F91EC06F00401610E826FF0
:1012E00091EC06F03BEF09F00101620E046F010E74
:1012F000056F000E066F000E076F59C100F15AC14D
:1013000001F15BC102F15CC103F109EC11F003BF13
:10131000D1EF09F00E0E2AEC05F0E8CF0CF10F0E1C
:101320002AEC05F0E8CF0DF1100E2AEC05F0E8CF1D
:101330000EF1110E2AEC05F0E8CF0FF152EC10F08F
:1013400059C104F15AC105F15BC106F15CC107F155
:1013500009EC11F0078216EC10F052EC10F0079235
:1013600016EC10F059C100F15AC101F15BC102F154
:101370005CC103F1079216EC10F0CC0E046FE00E86
:10138000056F870E066F050E076F09EC11F000C19F
:101390000CF101C10DF102C10EF103C10FF109EF12
:1013A0000AF00101800E006F1A0E016F060E026F27
:1013B000000E036F42C104F143C105F144C106F1BF
:1013C00045C107F109EC11F003AFEAEF09F000ECB9
:1013D00012F012000E0E2AEC05F0E8CF0CF10F0E01
:1013E0002AEC05F0E8CF0DF1100E2AEC05F0E8CF5D
:1013F0000EF1110E2AEC05F0E8CF0FF142C100F119
:1014000043C101F144C102F145C103F1078216EC69
:1014100010F00CC100F10DC101F10EC102F10FC1BC
:1014200003F112008251520A03E10E8219EF0AF011
:101430000E92078455C159F156C15AF157C15BF15B
:1014400058C15CF13EC142F13FC143F140C144F19A
:1014500041C145F14AC14CF14BC14DF107940EA079
:1014600050EF0AF0010165673DEF0AF066673DEF56
:101470000AF067673DEF0AF0686741EF0AF050EF46
:101480000AF074EC09F065C104F166C105F167C1A9
:1014900006F168C107F109EC11F003BF8AEF0BF008
:1014A00074EC09F00101000E046F000E056F010ECF
:1014B000066F000E076F37EC11F00401720E826F99
:1014C00091EC06F004012C0E826F91EC06F0A3EC77
:1014D00011F01D6771EF0AF00401200E826F74EFA6
:1014E0000AF004012D0E826F91EC06F024C182F403
:1014F0000401300E822791EC06F025C182F404012C
:10150000300E822791EC06F004012E0E826F91ECD2
:1015100006F026C182F40401300E822791EC06F019
:1015200027C182F40401300E822791EC06F00401F9
:101530006D0E826F91EC06F004012C0E826F91EC1F
:1015400006F042C100F143C101F144C102F145C1BD
:1015500003F10101A3EC11F0CFEC0FF00401480EF0
:10156000826F91EC06F004017A0E826F91EC06F026
:1015700004012C0E826F91EC06F059C100F15AC1A2
:1015800001F15BC102F15CC103F10101A3EC11F0B7
:10159000CFEC0FF00401630E826F91EC06F00401B2
:1015A0002C0E826F91EC06F059C100F15AC101F185
:1015B0005BC102F15CC103F101010A0E046F000E70
:1015C000056F000E066F000E076F18EC11F0000E8D
:1015D000046F120E056F000E066F000E076F37ECDA
:1015E00011F0A3EC11F01EC182F40401300E822729
:1015F00091EC06F01FC182F40401300E822791ECB9
:1016000006F020C182F40401300E822791EC06F02E
:1016100021C182F40401300E822791EC06F022C130
:1016200082F40401300E822791EC06F023C182F48B
:101630000401300E822791EC06F024C182F40401EB
:10164000300E822791EC06F004012E0E826F91EC91
:1016500006F025C182F40401300E822791EC06F0D9
:1016600026C182F40401300E822791EC06F027C1D6
:1016700082F40401300E822791EC06F00401730E0F
:10168000826F91EC06F004012C0E826F91EC06F053
:1016900000EC12F04CC100F14DC101F1EBEC0CF08B
:1016A0000EB256EF0BF00EA088EF0BF004012C0EDB
:1016B000826F91EC06F0200EF86EF76AF66A04016C
:1016C0000900F5CF82F491EC06F00900F5CF82F421
:1016D00091EC06F00900F5CF82F491EC06F00900D8
:1016E000F5CF82F491EC06F00900F5CF82F491EC8D
:1016F00006F00900F5CF82F491EC06F00900F5CF71
:1017000082F491EC06F00900F5CF82F491EC06F03A
:101710009BEC06F00E90C2EF0BF00401630E826F9B
:1017200091EC06F004012C0E826F91EC06F0C7ECF0
:101730000BF004012C0E826F91EC06F03AEC0CF0E9
:1017400004012C0E826F91EC06F0B6EC0CF0040153
:101750002C0E826F91EC06F00101F80E006FCD0E99
:10176000016F660E026F030E036FDCEC0BF00401D9
:101770002C0E826F91EC06F0CCEC0CF09BEC06F09A
:10178000C2EF0BF00301A26B0790CDEF0EF0D890E3
:101790000E0E2AEC05F0E8CF00F10F0E2AEC05F052
:1017A000E8CF01F1100E2AEC05F0E8CF02F1110E9E
:1017B0002AEC05F0E8CF03F10101000E046F000EE2
:1017C000056F010E066F000E076F37EC11F0A3ECEA
:1017D00011F01EC182F40401300E822791EC06F054
:1017E0001FC182F40401300E822791EC06F020C163
:1017F00082F40401300E822791EC06F021C182F4BC
:101800000401300E822791EC06F022C182F404011B
:10181000300E822791EC06F023C182F40401300ED1
:10182000822791EC06F024C182F40401300E822755
:1018300091EC06F025C182F40401300E822791EC70
:1018400006F004012E0E826F91EC06F026C182F4A0
:101850000401300E822791EC06F027C182F40401C6
:10186000300E822791EC06F004016D0E826F91EC30
:1018700006F01200120E2AEC05F0E8CF00F1130E6C
:101880002AEC05F0E8CF01F1140E2AEC05F0E8CFC0
:1018900002F1150E2AEC05F0E8CF03F101010A0E62
:1018A000046F000E056F000E066F000E076F18EC38
:1018B00011F0000E046F120E056F000E066F000E81
:1018C000076F37EC11F0A3EC11F01EC182F4040194
:1018D000300E822791EC06F01FC182F40401300E15
:1018E000822791EC06F020C182F40401300E822799
:1018F00091EC06F021C182F40401300E822791ECB4
:1019000006F022C182F40401300E822791EC06F029
:1019100023C182F40401300E822791EC06F024C129
:1019200082F40401300E822791EC06F004012E0EA1
:10193000826F91EC06F025C182F40401300E8227FB
:1019400091EC06F026C182F40401300E822791EC5E
:1019500006F027C182F40401300E822791EC06F0D4
:101960000401730E826F91EC06F012000A0E2AEC4D
:1019700005F0E8CF00F10B0E2AEC05F0E8CF01F1FD
:101980000C0E2AEC05F0E8CF02F10D0E2AEC05F062
:10199000E8CF03F1EBEF0CF0060E2AEC05F0E8CFF0
:1019A00000F1070E2AEC05F0E8CF01F1080E2AEC51
:1019B00005F0E8CF02F1090E2AEC05F0E8CF03F1BB
:1019C000EBEF0CF0010100EC12F007844AC100F1CA
:1019D0004BC101F107940101E80E046F800E056F01
:1019E000000E066F000E076F18EC11F0000E046F6A
:1019F000040E056F000E066F000E076F37EC11F036
:101A0000880E046F130E056F000E066F000E076F31
:101A100009EC11F00A0E046F000E056F000E066F40
:101A2000000E076F37EC11F0A3EC11F001011D67F8
:101A30001FEF0DF00401200E826F22EF0DF0040164
:101A40002D0E826F91EC06F024C182F40401300E59
:101A5000822791EC06F025C182F40401300E822722
:101A600091EC06F026C182F40401300E822791EC3D
:101A700006F004012E0E826F91EC06F027C182F46D
:101A80000401300E822791EC06F00401430E826FB0
:101A900091EC06F0120087C31EF188C31FF189C3C1
:101AA00020F18AC321F18BC322F18CC323F18DC3B2
:101AB00024F18EC325F190C326F191C327F10101D2
:101AC0004DEC12F0C5EC11F00101000E046F000E98
:101AD000056F010E066F000E076F18EC11F00E0E69
:101AE0000C6E00C10BF014EC05F00F0E0C6E01C172
:101AF0000BF014EC05F0100E0C6E02C10BF014ECA0
:101B000005F0110E0C6E03C10BF014EC05F004018E
:101B10007A0E826F91EC06F004012C0E826F91EC2C
:101B200006F00401350E826F91EC06F004012C0ED4
:101B3000826F91EC06F0C7EC0BF04AEF09F087C317
:101B40001EF188C31FF189C320F18AC321F18BC321
:101B500022F18CC323F18DC324F18EC325F190C3F0
:101B600026F191C327F101014DEC12F0C5EC11F003
:101B7000880E046F130E056F000E066F000E076FC0
:101B80000DEC11F0000E046F040E056F000E066FD1
:101B9000000E076F18EC11F00101E80E046F800EC3
:101BA000056F000E066F000E076F37EC11F00A0E7E
:101BB0000C6E00C10BF014EC05F00B0E0C6E01C1A5
:101BC0000BF014EC05F00C0E0C6E02C10BF014ECD3
:101BD00005F00D0E0C6E03C10BF014EC05F00401C2
:101BE0007A0E826F91EC06F004012C0E826F91EC5C
:101BF00006F00401360E826F91EC06F004012C0E03
:101C0000826F91EC06F0B6EC0CF04AEF09F087C356
:101C10001EF188C31FF189C320F18AC321F18BC350
:101C200022F18CC323F18DC324F18FC325F190C31E
:101C300026F191C327F101014DEC12F0C5EC11F032
:101C4000000E046F120E056F000E066F000E076F78
:101C500018EC11F001010A0E046F000E056F000E62
:101C6000066F000E076F37EC11F0120E0C6E00C1FC
:101C70000BF014EC05F0130E0C6E01C10BF014EC1C
:101C800005F0140E0C6E02C10BF014EC05F0150EED
:101C90000C6E03C10BF014EC05F004017A0E826F98
:101CA00091EC06F004012C0E826F91EC06F0040119
:101CB000370E826F91EC06F004012C0E826F91ECCE
:101CC00006F03AEC0CF04AEF09F087C31EF188C326
:101CD0001FF189C320F18AC321F18BC322F18CC388
:101CE00023F18DC324F18EC325F190C326F191C356
:101CF00027F101014DEC12F0C5EC11F0880E046FD4
:101D0000130E056F000E066F000E076F0DEC11F03D
:101D1000000E046F040E056F000E066F000E076FB5
:101D200018EC11F00101E80E046F800E056F000E33
:101D3000066F000E076F37EC11F0060E0C6E00C137
:101D40000BF014EC05F0070E0C6E01C10BF014EC57
:101D500005F0080E0C6E02C10BF014EC05F0090E34
:101D60000C6E03C10BF014EC05F004017A0E826FC7
:101D700091EC06F004012C0E826F91EC06F0040148
:101D8000380E826F91EC06F004012C0E826F91ECFC
:101D900006F0CCEC0CF04AEF09F081A88BEF0FF0C5
:101DA00007A844EF0FF00101800E006F1A0E016FBB
:101DB000060E026F000E036F3EC104F13FC105F134
:101DC00040C106F141C107F109EC11F003BF8BEFEF
:101DD0000FF0C9EC0FF03EC100F13FC101F140C16D
:101DE00002F141C103F1078216EC10F00CC104F1BD
:101DF0000DC105F10EC106F10FC107F1F80E006F1C
:101E0000CD0E016F660E026F030E036F09EC11F029
:101E10000E0E0C6E00C10BF014EC05F00F0E0C6EE4
:101E200001C10BF014EC05F0100E0C6E02C10BF0AA
:101E300014EC05F0110E0C6E03C10BF014EC05F060
:101E40000784010100EC12F04AC100F14BC101F11D
:101E500007940A0E0C6E00C10BF014EC05F00B0E8B
:101E60000C6E01C10BF014EC05F00C0E0C6E02C1EF
:101E70000BF014EC05F00D0E0C6E03C10BF014EC1E
:101E800005F007988BEF0FF007AA8BEF0FF0078490
:101E9000010100EC12F04AC100F14BC101F10794BD
:101EA000060E0C6E00C10BF014EC05F0070E0C6E64
:101EB00001C10BF014EC05F0080E0C6E02C10BF022
:101EC00014EC05F0090E0C6E03C10BF014EC05F0D8
:101ED000078455C100F156C101F157C102F158C143
:101EE00003F10794120E0C6E00C10BF014EC05F018
:101EF000130E0C6E01C10BF014EC05F0140E0C6EF9
:101F000002C10BF014EC05F0150E0C6E03C10BF0C2
:101F100014EC05F0079A0401805181197F0B0BE046
:101F20009EA809D014EE00F081517F0BE126E75006
:101F3000812B0F01AD6E16EF06F00CC100F10DC143
:101F400001F10EC102F10FC103F1000E046F000E8A
:101F5000056F010E066F000E076F37EC11F01DA123
:101F6000C8EF0FF01451D8B4C8EF0FF00CC100F156
:101F70000DC101F10EC102F10FC103F1000E046F9A
:101F8000000E056F0A0E066F000E076F37EC11F09A
:101F9000120001010C6B0D6B0E6B0F6B12001EC15A
:101FA00082F40401300E822791EC06F01FC182F406
:101FB0000401300E822791EC06F020C182F4040166
:101FC000300E822791EC06F021C182F40401300E1C
:101FD000822791EC06F022C182F40401300E8227A0
:101FE00091EC06F023C182F40401300E822791ECBB
:101FF00006F024C182F40401300E822791EC06F031
:1020000025C182F40401300E822791EC06F026C12E
:1020100082F40401300E822791EC06F027C182F48D
:102020000401300E822791EC06F0120001010053EA
:1020300005E1015303E1025301E1002BD9EC10F05B
:1020400000EC12F02C51006F2D51016F420E046F05
:102050004B0E056F000E066F000E076F18EC11F0A7
:1020600000C104F101C105F102C106F103C107F18C
:102070000CC100F10DC101F10EC102F10FC103F15C
:1020800007B247EF10F00DEC11F049EF10F009EC3A
:1020900011F000C10CF101C10DF102C10EF103C13B
:1020A0000FF1120000EC12F04CC100F14DC101F132
:1020B000060E2AEC05F0E8CF04F1070E2AEC05F035
:1020C000E8CF05F1080E2AEC05F0E8CF06F1090E7D
:1020D0002AEC05F0E8CF07F109EC11F000C118F186
:1020E00001C119F102C11AF103C11BF1290E046FDC
:1020F000000E056F000E066F000E076F18EC11F052
:10210000EE0E046F430E056F000E066F000E076F94
:102110000DEC11F018C104F119C105F11AC106F155
:102120001BC107F118EC11F000C110F101C111F150
:1021300002C112F103C113F1120E2AEC05F0E8CF2F
:1021400004F1130E2AEC05F0E8CF05F1140E2AEC89
:1021500005F0E8CF06F1150E2AEC05F0E8CF07F1FF
:102160000D0E006F000E016F000E026F000E036F68
:1021700018EC11F0180E046F000E056F000E066FBC
:10218000000E076F37EC11F010C104F111C105F119
:1021900012C106F113C107F10DEC11F06A0E046FC4
:1021A0002A0E056F000E066F000E076F09EC11F086
:1021B0001200BF0EFA6E200E2D6F2C6BD8900037D8
:1021C000013702370337D8B0EAEF10F02D2FDFEFD9
:1021D00010F02C072D070353D8B412000331070B5E
:1021E0008009326F03390F0B010F2C6F80EC5FF009
:1021F000336F2C0580EC5FF0335D335F2C6B323333
:10220000D8B02C272C3332A9FFEF10F033512C27F4
:10221000120025EC12F0D8B0120003510719286FF4
:10222000E8EC11F0D8900751031928AF800F120085
:10223000286B0CEC12F0D8A022EC12F0D8B01200EF
:10224000F7EC11F000EC12F01F0E296F38EC12F0D1
:102250000B35D8B0E8EC11F0D8A00335D8B0120097
:10226000292F26EF11F028B10FEC12F01200286B85
:1022700004510511061107110008D8A00CEC12F04A
:10228000D8A022EC12F0D8B01200086B096B0A6BD0
:102290000B6B38EC12F01F0E296F38EC12F007515F
:1022A0000B5DD8A460EF11F006510A5DD8A460EF71
:1022B00011F00551095DD8A460EF11F00451085DDB
:1022C000D8A073EF11F00451085F0551D8A0053D67
:1022D000095F0651D8A0063D0A5F0751D8A0073D07
:1022E0000B5FD8900081292F4DEF11F028B10FEC32
:1022F00012F0286B0CEC12F0D8903CEC12F0075165
:102300000B5DD8A490EF11F006510A5DD8A490EFB0
:1023100011F00551095DD8A490EF11F00451085D4A
:10232000D8A09FEF11F0003F9FEF11F0013F9FEF0A
:1023300011F0023F9FEF11F0032BD8B4120028B127
:102340000FEC12F012000101286B0CEC12F0D8B067
:10235000120041EC12F0200E296F003701370237CE
:10236000033711EE27F00A0E2A6FE7360A0EE75CF4
:10237000D8B0E76EE5522A2FB5EF11F0292FADEF57
:1023800011F028B11D81D890120001010A0E286FAA
:10239000200E296F11EE1DF028512A6F0A0ED890D9
:1023A000E652D8B0E726E7322A2FD0EF11F00333F8
:1023B000023301330033292FCAEF11F0E750FF0F2A
:1023C000D8A00335D8B012001DB10FEC12F01200E6
:1023D000045100270551D8B0053D01270651D8B05A
:1023E000063D02270751D8B0073D032712000051D0
:1023F000086F0151096F02510A6F03510B6F1200F0
:102400000101006B016B026B036B12000101046B95
:10241000056B066B076B12000335D8A01200035141
:10242000800B001F011F021F031F003F1FEF12F050
:10243000013F1FEF12F0023F1FEF12F0032B282B7A
:10244000032512000735D8A012000751800B041F86
:10245000051F061F071F043F35EF12F0053F35EF3C
:1024600012F0063F35EF12F0072B282B072512003C
:102470000037013702370337083709370A370B3778
:1024800012001D6B1E6B1F6B206B216B226B236B6D
:10249000246B256B266B276B12001E510F0B1E6FD2
:1024A0001F510F0B1F6F20510F0B206F21510F0B6E
:1024B000216F22510F0B226F23510F0B236F2451D9
:1024C0000F0B246F25510F0B256F26510F0B266F15
:0824D00027510F0B276F1200CA
:10BF0000E844F926000C160C2B0C3F0C520C640C68
:10BF1000760C860C960CA50CB30CC10CCF0CDC0C6B
:06BF2000E80CF40C000C1B
:00000001FF
